:0800000000008A110A12182AFF
:06000A0001308316031310
:10001000860002308312031386000D2240210A302D
:10002000FF0000308921072283120313AA00313A0E
:10003000031939282A08323A03193B282A08333A87
:1000400003193D282A08343A03193F282A08353A6B
:10005000031946282A08703A031937282A08783ADB
:10006000031951282A087A3A03194D285428F621F1
:100070005428F0215428E5215428D2215428CC2199
:100080000A30FF0000308921B9215428CC210A30E0
:10009000FF0000308921B2215428831203138614F3
:1000A000542883120313861002308312031386062A
:1000B0000A30FF0000308921132808000030831225
:1000C0000313A2002E30FC002208FD000030FE00C9
:1000D0000230FF00E030B420831203132E08080022
:1000E000003083120313A2002D30FC002208FD0013
:1000F0000030FE000330FF00E030B4208312031311
:100100002D0808005130FE000030FF00E0300621CD
:100110000800003083120313A1002C30FC002108DA
:10012000FD000030FE000130FF00E030B4208312FB
:1001300003132C080800003083120313A1002B3096
:10014000FC002108FD000030FE000030FF00E03020
:10015000B420831203132B0808006030FE00003027
:10016000FF00E0300621080083120313A4007F087B
:10017000A5007E08A8007D08A7007C08A6006F21C6
:1001800069218312031324085921692177218312DD
:100190000313A90029080319D02854210030052988
:1001A0008312031325085921692177218312031330
:1001B000A50025080319DF285421003005296521F1
:1001C000692183120313A40A240859216921772184
:1001D00083120313A40024080319F12854210030CA
:1001E00005295D2183120313A400FD002608FE00EB
:1001F0002708FF0028088A110A12AC228A110A1265
:100200007F216921732169210130080083120313C2
:10021000A0007F08A1007E08A2006F21692183123F
:100220000313200859216921772183120313A000A9
:10023000200803191E29542100303F29831203137B
:10024000210859216921772183120313A000200876
:1002500003192D29542100303F298312031322084A
:1002600059216921772183120313A0002008031963
:100270003C29542100303F297321692101300800B5
:1002800018308316031387049401941708308312DF
:1002900003139400941683160313910131309300D5
:1002A000831203138C110800732169216630F92130
:1002B000080083120313930008008316031391159B
:1002C0006921831203131308080083160313911482
:1002D0000800831203138C1D69298C1108008316F2
:1002E0000313111408008316031311150800831655
:1002F0000313111B7D2900307E290130080083166D
:100300000313911611160800831603139112111688
:10031000080083120313A0007F08A10083120313B7
:100320002008803E803E031D972901302102031CD6
:10033000B129FF3083120313A2000F30A3008312F0
:100340000313220823040319AA29FF30A207031C60
:10035000A3039F29FF3083120313A107031CA003EB
:100360008E2908008A110A1270208A110A12F921B6
:1003700008008A110A1270208A110A1283120313CC
:10038000A0008A110A125E208A110A12F921831232
:1003900003132008F92108008A110A1282208A1109
:1003A0000A1208008A110A1289208A110A1283127D
:1003B0000313A000803A031DE0293130F921E4291C
:1003C000831203132008F92108003C30F9218A1117
:1003D0000A129B208A110A12F9213E30F9210800E5
:1003E0008A110A12AD208A110A1208006F30F92111
:1003F000080083120313A000831203130C1EFC29B0
:100400008312031320088312031399000800831238
:1004100003138C1E072A1A08080081308316031361
:10042000990024309800903083120313980008003C
:10043000EC30FE000230FF0080308A110A12CB221D
:100440008A110A1283120313B0007F08AF00EE3046
:10045000B1000230B200831203132F08B30030083A
:10046000B400FF30AF07031CB00333083404031992
:10047000A82A04303107B300B401B40D3208B40720
:100480003308FE003408FF0080308A110A12CB22A4
:100490008A110A1283120313B6007F08B5003108CF
:1004A000FE003208FF0080308A110A12CB228A1126
:1004B0000A1283120313B800B4007F08B700B30018
:1004C00002303107B300B401B40D3208B407330869
:1004D000FE003408FF0080308A110A12CB228A11F4
:1004E0000A1283120313B400BA007F08B300B900E4
:1004F000831203133508B9003608BA00FF30B50778
:10050000031CB60339083A040319A12A3708FE0070
:100510003808FF0080308A110A12B8228A110A12A4
:1005200083120313B900330884008313341883172C
:1005300039088000B70A0319B80AB30A0319B40AC4
:10054000782A063083120313B1070318B20A2B2A44
:100550008A110A1205280800003A0319B02A080077
:100560007E08840083137F1883177D0880000800AD
:10057000003A0319BF2A803A0319C62A00347E08BC
:10058000840083137F188317000808007F088A00FF
:100590007E0882000800003A0319D32A803A031922
:1005A000DD2AFF0100347E08840083137F1883173F
:1005B0000008FF00840A000808008A110A12C622F7
:1005C000FD00FE0FFF03FF0A8A110A12C622FC007B
:1005D0007D08FF007C08080001340034F434023444
:0A05E0003B340034013400340034D1
:00000001FF
